:100000000C94A0000C94BE000C94BE000C94BE0096
:100010000C94BE000C94BE000C94BE000C94BE0068
:100020000C94BE000C94BE000C94780A0C94BE0094
:100030000C94BE000C94BE000C94BE000C94BE0048
:100040000C94BE000C94BE000C94BE000C94BE0038
:100050000C9461010C94BE000C94BE000C946704D7
:100060000C94BE000C94DB010C94BE000C94BE00FA
:100070000C94BE000C94DA000C94BE000C94BE00EC
:100080000C94BE000C94BE000C94BE000C94BE00F8
:100090000C94BE000C94BE000C94BE000C94BE00E8
:1000A0000C94BE000C94BE000C94BE001201000221
:1000B00002000020EB0318200010000000010902DC
:1000C0004300020100803209040000010202010025
:1000D000052400100105240103010424020605245F
:1000E000060001070583032000FF09040100020A3E
:1000F0000000000705810220000007050202200021
:10010000000C03410054004D0045004C0022034107
:1001100000560052002000550053004200200043CA
:1001200000440043002000440045004D004F000CF7
:100130000331002E0030002E0030000403090400BB
:1001400011241FBECFEFDAE0DEBFCDBF81E011E0AA
:10015000A0E0B1E0E0E9F8E202C005900D92AC3217
:10016000B107D9F712E0ACE2B1E001C01D92AF3C9B
:10017000B107E1F70E94BA040C9446140C940000F5
:1001800089ED86BD14BC84E085BD81E080936E005E
:10019000089581E480937C0010927B00EAE7F0E010
:1001A00080E8808380E980838EEC808383E3809382
:1001B0007E0008951F920F920FB60F9211248F9315
:1001C0009F9380913F01882369F4809178009091FA
:1001D00079009093AD018093AC0181E080933F0161
:1001E00081E447C080913F01813069F480917800BB
:1001F000909179009093AF018093AE0182E080935B
:100200003F0184E436C080913F01823069F48091DF
:100210007800909179009093B1018093B00183E0D0
:1002200080933F0185E425C080913F01833091F4A4
:1002300080917800909179009093B3018093B201FE
:1002400084E080933F0187EC80937C0080E2809380
:100250007B0013C080913F01843079F48091780055
:10026000909179009093B5018093B40110923F0171
:1002700080E480937C0010927B008EEC80937A0067
:100280009F918F910F900FBE0F901F901895109215
:10029000850010928400E6E8F0E02FEF33E0318330
:1002A00020838FEF809380008AE0809381003183E8
:1002B000208310928200EFE6F0E0808181608083ED
:1002C00008951F920F920FB60F9211241092800082
:1002D0001092810010928500109284000F900FBE42
:1002E0000F901F901895813049F48FEF93E0861B93
:1002F000970B90938900809388000895823049F489
:100300008FEF93E0861B970B90938B0080938A006E
:100310000895833041F48FEF93E0861B970B909301
:100320008D0080938C00089520913D0140917F01C4
:1003300090E030E0241B3109AC01429FC001439F93
:10034000900D529F900D112464EB70E00E94AA0F53
:100350009B0180917F01280F311DC90108951F93D2
:10036000182F862F0E949401BC01812F0E947301D7
:100370001F91089580538A3008F087500895809126
:1003800080018F5F8093800108951F939C0180916D
:10039000BA01882371F01091E90081E08093E900AF
:1003A0008091E80085FFFCCFC9010E94C805109329
:1003B000E9001F9108951F920F920FB60F9211241A
:1003C0001F932F933F934F935F936F937F938F93DD
:1003D0009F93AF93BF93EF93FF938091BA018823CC
:1003E000E9F01091E90081E08093E90060E08091FC
:1003F000C80087FF09C05F9AE62FF0E08091CE0029
:10040000EC5AFE4F80836F5F8091E80085FFEFCF4D
:1004100084E591E00E94C8051093E900FF91EF91F7
:10042000BF91AF919F918F917F916F915F914F910C
:100430003F912F911F910F900FBE0F901F90189515
:100440001F93682F8091BA01882379F01091E900F9
:1004500081E08093E9008091E80085FFFCCF84E58E
:1004600091E00E94C8051093E9001F9108950E9431
:10047000010F8091BA01882369F00E947F058823CB
:1004800029F408950E949F050E941B0C8091B601DB
:100490008823C1F70895EF92FF920F93CF93DF93D4
:1004A00009B100950170499B0E5F4D9B0C5F629BEB
:1004B000085F7F9B005F7E9B005E2091AC013091C6
:1004C000AD014091AE015091AF016091B0017091CA
:1004D000B101E090B201F090B301C091B401D091AC
:1004E000B5018DB79EB740970FB6F8949EBF0FBE6B
:1004F0008DBFEDB7FEB7319684E591E0ADB7BEB7DD
:1005000012969C938E93119780E091E0938382835F
:1005100004831582378326835187408773876287D8
:10052000F586E486D787C6870E9446108DB79EB7AA
:1005300040960FB6F8949EBF0FBE8DBF88E190E045
:100540000E942002DF91CF910F91FF90EF900895CC
:10055000809184018C3409F499C08D3430F4833453
:10056000B9F1843409F046C10AC0833509F444C0A6
:10057000863509F43DC1823509F03CC160C09091D7
:100580008501892F90FF02C05C9A01C05C9881FFB1
:1005900002C05E9A01C05E9882FF02C05F9A01C0ED
:1005A0005F9883FF02C02C9A01C02C9884FF02C080
:1005B0002D9A01C02D9885FF02C02E9A01C02E9859
:1005C00086FF02C0469A01C0469897FFC9C093C0F3
:1005D0008091850180FF02C02F9A01C02F9881FF72
:1005E00002C02B9A01C02B9882FF02C02A9A01C038
:1005F0002A9883FF90C05AC080918501803309F406
:100600005DC0813309F45EC0823309F45FC0833377
:1006100009F460C0843309F461C0853309F462C011
:10062000863309F463C0873309F465C08435B1F1BA
:100630008634C1F18934F1F18335C1F1DBC0809199
:100640008501803309F46FC0813309F470C08233AF
:1006500009F471C0833309F472C0843309F473C0A0
:10066000853309F474C0863309F475C0873309F4FF
:1006700077C0843509F447C0863409F448C089340A
:1006800009F44DC0833509F446C0B4C0809185019A
:100690008E3499F580918601813011F42F9AAAC089
:1006A000823011F42B9AA6C0833011F4299AA2C08B
:1006B000843011F42A9A9EC0853011F45C9A9AC055
:1006C000863011F45E9A96C0873011F45F9A92C01A
:1006D000883011F42C9A8EC0893011F42D9A8AC07A
:1006E0008A3011F42E9A86C08B3011F4469A82C05B
:1006F0008C3009F07FC0479A7DC0863499F580918F
:100700008601813011F42F9875C0823011F42B9836
:1007100071C0833011F429986DC0843011F42A9887
:1007200069C0853011F45C9865C0863011F45E981C
:1007300061C0873011F45F985DC0883011F42C9847
:1007400059C0893011F42D9855C08A3011F42E9873
:1007500051C08B3011F446984DC08C3009F04AC01E
:10076000479848C0843509F045C090918601913082
:1007700019F485B180582EC0923019F485B198E0F3
:1007800028C0933019F485B192E023C0943011F45D
:1007900085B11FC0953019F48BB190E104C096303B
:1007A00029F48BB190E489278BB924C0973019F4D0
:1007B0008BB18058F9CF983019F485B190E109C018
:1007C000993019F485B190E204C09A3029F485B1CA
:1007D00090E4892785B90EC09B3021F488B190E45C
:1007E000892704C09C3031F488B1805888B902C090
:1007F0000E944B028DE0809354018AE08093550162
:100800008EE38093560183E090E00E9420021092D4
:100810007D0108959FEF94B980EC87B980ED8AB986
:1008200080E48DB910BA15B88FE388B98FE28BB91F
:100830008FEB8EB991BB0E94130C10925201109253
:10084000510110923F010E94C90085B7806885BFA1
:1008500085B7806885BF85B7806885BF85B78068A4
:1008600085BF85B7806885BF10927D0189ED86BD03
:1008700014BC84E085BD81E080936E00E2EEF0E080
:100880008081846080838091810183608093810175
:100890008EEF95E06FE975E00E94FA0F08958AE007
:1008A00090E7FC018491EBE0F0E73491ECE0F0E7B5
:1008B0002491EDE0F0E794918C3231F4313121F460
:1008C0002C3211F4923211F00E94BA0408951F9252
:1008D0000F920FB60F9211242F933F934F935F9374
:1008E0006F937F938F939F93AF93BF93EF93FF93F8
:1008F00089ED86BD809140019091410101969093D0
:100900004101809340018091420190914301019601
:10091000909343018093420180914401909145015D
:1009200001969093450180934401809146019091F6
:1009300047010196909347018093460180914801B9
:1009400090914901019690934901809348010E943A
:100950003B0CFF91EF91BF91AF919F918F917F9150
:100960006F915F914F913F912F910F900FBE0F901C
:100970001F901895E7EDF0E080818160808388E02A
:100980008AB90E941D0580E090E0089513BE83B7E8
:10099000856083BF8895089513BE83B7816083BF48
:1009A0008895089513BE83B7836083BF88950895A3
:1009B00013BE83B7876083BF8895089513BE83B73E
:1009C0008D6083BF8895089513BE83B78F6083BF02
:1009D000889508958091C50084608093C5008091BA
:1009E000C70080FFFCCF8091C50081608093C50067
:1009F0008091C500877F8093C50008958091C500D0
:100A000088608093C5008091C70081FFFCCF8091F2
:100A1000C5008E7F8093C5008091C5008B7F809339
:100A2000C500089508950E948C0B0E943702FBCFE9
:100A30000E948F0B0E940A0408950E9418050E94CC
:100A4000130508958091CF029091D002A091D10218
:100A5000B091D20285559A4AAA4AB54569F41092D6
:100A6000CF021092D0021092D1021092D202E091E5
:100A70001901F0911A010995089585E59AEAAAEA03
:100A8000B5E58093CF029093D002A093D102B093AA
:100A9000D202A8958091600080618093600088E018
:100AA00080936000FFCF8091C8008078089589E12D
:100AB00090E09093CD008093CC00E8ECF0E0808152
:100AC0008260808386E08093CA00E9ECF0E0808158
:100AD0008861808381E00895282F8091C80085FF78
:100AE000FCCF2093CE00822F08958091C80087FF0D
:100AF000FCCF8091CE0008951092B60108958091A8
:100B0000B6018823B9F482E08093E9008091E8007F
:100B100082FF10C08091F2008093B601882351F4C7
:100B20008091E8008B7F8093E8008091E8008F77C8
:100B30008093E8008091B601811181E0089582E000
:100B40008093E9008091B601882319F40E947F0503
:100B5000FBCF9091F1008091B60181508093B60156
:100B6000882351F48091E8008B7F8093E800809186
:100B7000E8008F778093E800892F08958091E8003E
:100B800090E025E0969587952A95E1F78170089584
:100B9000FC0181E08093E900262F19C08091E800D4
:100BA00085FFFCCF04C081918093F100215080919A
:100BB000E80085FF02C02223B1F78091E8008E7F14
:100BC0008093E8008091E8008F778093E8002223EB
:100BD00029F7862F90E08F719070892B71F48091A6
:100BE000E80085FFFCCF8091E8008E7F8093E800CD
:100BF0008091E8008F778093E8000895DF93CF938A
:100C000000D0CDB7DEB79A838983CE01019661E02B
:100C10000E94C80589819A810F900F90CF91DF9132
:100C20000895E8EDF0E080818F778083808180688F
:100C300080838081806180838081816080837894DB
:100C400008958091D80080628093D80082B7807F19
:100C500082BF82B78A6482BF82E089BD09B400FE88
:100C6000FDCF8091D8008F7D8093D8008091E000E7
:100C70008E7F8093E0008091E000877F8093E0008A
:100C80008091E20081608093E2008091E2008860C0
:100C90008093E20078940E94CB06089580912C0105
:100CA000882371F48091D90080FF0AC08091D80018
:100CB00080688093D80081E080932C010E942106F7
:100CC00080913B0190913C0190FF10C080913B01CD
:100CD00090913C019E7F90933C0180933B0181E089
:100CE0008093EA001092EA001092BA011092E90093
:100CF0008091E80083FF02C00E9447080895909108
:100D0000EB0091609093EB008093EC008091ED00FC
:100D10008270862B8093ED008091ED00826080933D
:100D2000ED008091EE00881F8827881F089590911C
:100D3000F40080E090FD06C08F5F873011F096953B
:100D4000F9CF80E00895FB018093E90004C0819110
:100D50008093F10041508091E80085FF02C0442358
:100D6000B1F7842F0895FB018093E90004C08091BE
:100D7000F100819341508091E80085FF02C0442337
:100D8000B1F7842F08958093E900EBEEF0E08081C5
:100D90008062808308951092E9008091EB0080FFCB
:100DA00002C080E008951092E90082E060E20E94B3
:100DB0007F06089580E008958091E800877F809302
:100DC000E80080914A018093F10080914B0180936B
:100DD000F10080914C018093F10080914D0180934E
:100DE000F10080914E018093F10080914F0180933A
:100DF000F100809150018093F1008091E8008E7F96
:100E00008093E8008091E80080FFFCCF8091E800AB
:100E100082FFFCCF8091E8008B7F8093E800809177
:100E2000E8008F778093E80008958091E800877F3D
:100E30008093E8008091E80082FFFCCF8091F10070
:100E400080934A018091F10080934B018091F100E1
:100E500080934C018091F10080934D018091F100CD
:100E600080934E018091F10080934F018091F100B9
:100E7000809350018091E8008B7F8093E8008091FF
:100E8000E8008F778093E8008091E8008E7F809360
:100E9000E8008091E80080FFFCCF20914A0130916A
:100EA0004B0140914C0150914D0156954795379516
:100EB000279584E0220F331F441F551F8A95D1F7D1
:100EC00060E072E18AE790E00E94BD0F215030405F
:100ED0003093CD002093CC0008959091E800977F47
:100EE0009093E8009091E8009E7F9093E8008093B3
:100EF0007E018091E80080FFFCCF08952091810160
:100F00003091820180912F019091300182179307D7
:100F100011F480E008953093300120932F0183E095
:100F20008093E9008091E80085FD02C081E008958A
:100F300081EA8093F10080E28093F1001092F10049
:100F40001092F1001092F1001092F10082E0809373
:100F5000F1001092F100809181018093F100809165
:100F600082018093F1008091E8008E7F8093E800F9
:100F70008091E8008F778093E80081E00895809168
:100F8000E800877F8093E8008091E8008E7F80935F
:100F9000E80081E080932E018091E80080FFFCCF83
:100FA0000895DF93CF9300D0CDB7DEB72091F10045
:100FB0009091F1008132A9F429839A83623239F049
:100FC000633251F06032A9F40E94150710C0898184
:100FD0009A810E946D070BC089819A810E94BF0788
:100FE00006C0813A31F4613221F40E94DC0681E0CE
:100FF00001C080E00F900F90CF91DF910895FF9294
:101000000F931F9309EE10E083E0F801808381ECD9
:1010100060E20E947F0681E0F801808381E860E25F
:101020000E947F0622E0F22EF801F08280E860E262
:101030000E947F06EAEEF0E088E080831082F08272
:10104000108284E0808310821F910F91FF90089599
:1010500009B400FC0BC082B7807F82BF82B78A646C
:1010600082BF82E089BD09B400FEFDCF8091D80027
:101070008F7D8093D80080913101813039F4809147
:10108000E00082608093E000109231010895DF93C8
:10109000CF9300D0CDB7DEB78091E8008B7F8093EF
:1010A000E8009091F10090933A016091F100663070
:1010B000F9F0673068F4613009F41CC1613008F45C
:1010C00098C1633009F450C1653009F0FDC1D6C044
:1010D000693009F4F5C06A3020F4683009F0F4C1D1
:1010E000B0C06A3009F4C1C16B3009F0EDC1DBC199
:1010F000903809F0A3C0109232016091F100809104
:10110000F100813019F0823089F406C082E18093C9
:10111000BB018CEA90E005C083E48093BB018EEBB9
:1011200090E09093BD018093BC0105C00E94DA0657
:10113000882309F4CEC18091F1008091F100809163
:10114000F10089838091F1008A838091E800877F94
:101150008093E80029813A818091BB0190E0821759
:10116000930758F48F719070892B21F481E080935C
:10117000320105C01092320102C02093BB01809160
:10118000E8008F7E8093E8002091BC013091BD0182
:101190004091BB0122C08091E80084FF03C0F901A7
:1011A00090E00FC08091E80080FFF5CFF8CF542F7A
:1011B0005150903249F09F5F84918093F1003196B5
:1011C000452F9F01442399F78091E80084FD12C0C8
:1011D0008091E8008E7F8093E800442339F42093C7
:1011E000BC013093BD011092BB010AC08091E800A0
:1011F00084FFD8CF2093BC013093BD014093BB0145
:1012000080913201813069F48091E80084FD09C049
:101210008091E80080FFFCCF8091E8008E7F809372
:10122000E8008091E80084FFFCCF8091E8008F7E89
:101230008093E8008091E8008B7F53C1892F66E09E
:101240002FC19038C1F48091E800877F8093E80037
:101250008091BA018093F1008091E8008E7F8093A5
:10126000E8008091E8008F778093E8008091E800A3
:1012700082FFFCCF0AC1892F68E012C19923E9F4EB
:101280009091F1008091E3009F778078982B909364
:10129000E3008091E800877F8093E8008091E80078
:1012A0008E7F8093E8008091E80080FFFCCF8091E2
:1012B000E30080688093E30016C1892F65E0F0C0E9
:1012C0009923A9F49091F100923008F002C1809125
:1012D000E800877F8093E8009093BA018091E8004E
:1012E0008E7F8093E800892F0E94FF07FCC0892F22
:1012F00069E0D6C09330A8F5992309F441C0913034
:1013000009F4E7C08091F1009091F100882309F081
:10131000E0C0E091F100EF77E093E9008091EB000D
:1013200080FF61C0EE23B1F08091EB00806180937B
:10133000EB0081E090E00E2E02C0880F991F0A9406
:10134000E2F78093EA001092EA008091EB00886057
:101350008093EB001092E900F0E0ED5CFE4F10820C
:1013600039C0892F61E09CC0933008F03FC09130B4
:1013700009F4AFC0913020F0923009F0AAC003C048
:101380008091F100A6C08091F1009091F100882336
:1013900009F09FC0E091F100EF7751F48091EB00EC
:1013A00080628093EB008091E800877F8093E80063
:1013B000E093E9008091EB0080FF15C08091EB0085
:1013C00080628093EB001092E900F0E0ED5CFE4F4C
:1013D00081E080838091E800877F8093E80080919E
:1013E000E8008E7F7EC01092E90073C0892F63E011
:1013F00057C0892F80588330A8F58091F1008091E3
:10140000F100E091F100913861F0923891F090385C
:1014100009F05FC08091E800877F8093E80081E059
:1014200013C08091E800877F8093E8001092F1005C
:101430000DC08091E800877F8093E800F0E0EF77AF
:10144000F070ED5CFE4F80818093F1001092F1000E
:101450008091E8008E7F8093E8008091E80082FF11
:10146000FCCF13C0892F60E01BC09138B9F4809184
:10147000E800877F8093E8008091E8008E7F80936A
:10148000E8008091E80082FFFCCF8091E8008B7F2C
:101490008093E8008091E8008F7723C0892F6AE06D
:1014A0000E94D10720C09130F1F48091E800877F3D
:1014B0008093E8008091E8008E7F8093E80080911F
:1014C000E80080FFFCCF0FC0892F0E94D10788233E
:1014D00051F48091EB0080628093EB008091E800F2
:1014E000877F8093E8000F900F90CF91DF91089550
:1014F0001F920F920FB60F9211242F933F934F9389
:101500005F936F937F938F939F93AF93BF93EF936B
:10151000FF938091DA0080FF31C08091D80080FF76
:101520002DC08EEF8093DA008091D90080FF19C022
:1015300081E080932C0180913B0190913C0182607D
:1015400090933C0180933B018091E20088608093FE
:10155000E2000E9421068091E0008E7F8093E000EF
:101560000DC010922C011092BA0180913B01909114
:101570003C01846090933C0180933B018091E100A9
:1015800082FF09C08091E20082FF05C08BEF80934B
:10159000E1000E94BF018091E10080FF29C080919D
:1015A000E20080FF25C081E080932D018FEE8093C3
:1015B000E10080913B0190913C01806290933C015D
:1015C00080933B018EEF8093E1008091E200806187
:1015D0008093E2008091E2008F7D8093E200809111
:1015E000D80080628093D80089B58D7F89BD19BCF1
:1015F0008091E10084FF47C08091E20084FF43C0F6
:1016000009B400FC0BC082B7807F82BF82B78A64B6
:1016100082BF82E089BD09B400FEFDCF8091D80071
:101620008F7D8093D8009FEE9093E10080912D01F3
:10163000882349F18091E20080628093E2008091EA
:10164000E20088608093E2009093E1008091E200E4
:101650008F7E8093E20080913B0190913C018064F9
:1016600090933C0180933B018091E20081608093E4
:10167000E2008091E20080628093E2008091E200CB
:1016800088608093E2008091E10085FF1CC080911A
:10169000E20085FF18C010922D018091E2008F7E3C
:1016A0008093E2008FED8093E1008091E2008F7DD6
:1016B0008093E20080913B0190913C01806890937F
:1016C0003C0180933B018091E10083FF14C0809135
:1016D000E20083FF10C01092B90187EF8093E10010
:1016E0000E94CB0680913B0190913C0191609093C8
:1016F0003C0180933B01FF91EF91BF91AF919F918E
:101700008F917F916F915F914F913F912F910F90AA
:101710000FBE0F901F9018950E944E0608950E94CC
:1017200011061092B90108952FEF33E0309387002E
:1017300020938600E0E8F0E020812068208323E108
:1017400020938100109282009093890080938800FA
:1017500008952FEF33E03093870020938600E0E870
:10176000F0E020812062208323E120938100109209
:10177000820090938B0080938A0008952FEF33E0CE
:101780003093870020938600E0E8F0E02081286015
:10179000208323E1209381001092820090938D009A
:1017A00080938C000895DC018C914FEF5FEF482708
:1017B000842F82958427082E869586958025082E6D
:1017C000869580258770042E452F869507948795EA
:1017D000502D4827069487955025482721E030E072
:1017E0001DC0FD01E20FF31F80814827842F8295E1
:1017F0008427082E869586958025082E8695802537
:101800008770042E452F869507948795502D48277D
:1018100006948795502548272F5F3F4F2617370797
:1018200004F3CA0108951092BF021092BE0281E033
:101830008093C40208952091BE023091BF02F90145
:10184000E051FE4F80832F5F3F4F3093BF022093C4
:10185000BE028091BE029091BF028436910530F0A5
:1018600083E690E09093BF028093BE021092C10283
:101870001092C00208958091C0029091C102019619
:101880009093C1028093C0028091C0029091C102E6
:10189000039758F01092BF021092BE021092C1023C
:1018A0001092C00281E08093C40208956091BA0250
:1018B0007091BB028091F0014FEF5FEF4827842FBA
:1018C00082958427082E869586958025082E8695F4
:1018D00080258770042E452F869507948795502D77
:1018E0004827069487955025482721E030E01DC001
:1018F000F901E051FE4F80814827842F829584278B
:10190000082E869586958025082E869580258770D9
:10191000042E452F869507948795502D48270694C9
:101920008795502548272F5F3F4F2617370704F329
:101930008091BA029091BB0281E090E00895282F37
:10194000332727FD309520FF02C05C9A01C05C98C8
:1019500021FF02C05E9A01C05E9822FF02C05F9A1A
:1019600001C05F9823FF02C02C9A01C02C9824FF6D
:1019700002C02D9A01C02D9825FF02C02E9A01C0E9
:101980002E9826FF02C0469A01C0469887FF02C0E3
:10199000479A01C04798772767FD709560FF02C09E
:1019A0002F9A01C02F9861FF02C02B9A01C02B987B
:1019B00062FF02C0299A01C0299863FF02C02A9AD7
:1019C00001C02A9864FF02C0289A01C0289865FFC8
:1019D00002C0769A089576980895CF92DF92EF929A
:1019E000FF920F931F93CF93DF9379B1709571702E
:1019F000499B7E5F4D9B7C5F629B785F7F9B705FA6
:101A00007E9B705EA3B1AA1FAA27AA1F1B99AE5F77
:101A10001999AC5F1A99A85F1899A05F6699A05EA2
:101A200089B190E064E0969587956A95E1F7682F13
:101A300061704E996E5F4F996C5F1C99685F1D993C
:101A4000605F1E99605E3699605C3799605890912E
:101A5000C3029330C9F0943020F4913009F078C17A
:101A600007C0953009F4E7C0963009F071C1ECC0A9
:101A7000909354029093550282E0809356027093A3
:101A8000570210925802DDC081E080935402909377
:101A900055028091F501E82EFF248091F301870122
:101AA000000F111F00935602C0E0D0E043E050E069
:101AB00024E030E0C82EDD24B1E0B5C0CE018C0DAD
:101AC0009D1D8530910509F474C086309105ACF4F4
:101AD0008230910509F446C08330910534F40097B3
:101AE00019F1019709F09AC02CC08330910509F4CF
:101AF00046C0049709F092C04FC08830910509F4A0
:101B000073C08930910544F48630910509F45AC0B8
:101B1000079709F083C05FC08930910509F46DC053
:101B20000A9709F07BC072C08091AC019091AD0121
:101B3000FA01EC5AFD4F90838091AC019091AD0178
:101B40000CC08091AE019091AF01FA01EC5AFD4FAB
:101B500090838091AE019091AF01F901EC5AFD4F55
:101B600080835CC08091B0019091B101FA01EC5A80
:101B7000FD4F90838091B0019091B101EECF8091A3
:101B8000B2019091B301FA01EC5AFD4F908380911C
:101B9000B2019091B301E1CF8091B4019091B50170
:101BA000FA01EC5AFD4F90838091B4019091B501F8
:101BB000D4CFFA01EC5AFD4F1082F901EC5AFD4FD7
:101BC00070832CC0FA01EC5AFD4F6083F901EC5A86
:101BD000FD4FA08323C080918900FA01EC5AFD4F8C
:101BE000808380918800B9CF80918B00FA01EC5AF4
:101BF000FD4F808380918A00B0CF80918D00FA01E3
:101C0000EC5AFD4F808380918C00A7CFFA01EC5AEB
:101C1000FD4FB083F901EC5AFD4F108221964E5FC3
:101C20005F4F2E5F3F4FCE15DF050CF447CFB80155
:101C30006D5F7F4F8DC08091F4016091F5010E942E
:101C40009F0C65E070E084C081E080935402909323
:101C500055028091F201809356028091F3018093A6
:101C600057028091F401809358028091F50180938E
:101C700059028091F301873099F0883020F4863042
:101C800009F064C006C0883041F1893009F05EC0B7
:101C900041C08091F4016091F5010E949F0C56C0F3
:101CA0002091F4013091F501922F80E0830F911D76
:101CB0002FEF33E03093870020938600209180003F
:101CC00020682093800023E12093810010928200FD
:101CD000909389008093880039C02091F40130915D
:101CE000F501922F80E0830F911D2FEF33E03093A9
:101CF000870020938600209180002062209380003E
:101D000023E1209381001092820090938B008093B6
:101D10008A001CC02091F4013091F501922F80E0DF
:101D2000830F911D2FEF33E03093870020938600BF
:101D30002091800028602093800023E1209381007F
:101D40001092820090938D0080938C0066E070E08A
:101D5000809154022FEF3FEF2827822F8295822710
:101D6000082E869586958025082E86958025877075
:101D7000022E232F869507948795302D28270694C9
:101D800087953025282741E050E01DC0FA01EC5A24
:101D9000FD4F80812827822F82958227082E8695E5
:101DA00086958025082E869580258770022E232F04
:101DB000869507948795302D28270694879530259A
:101DC00028274F5F5F4F4617570704F3FB01EC5A74
:101DD000FD4F2083CB010196232F330F330BFC01E2
:101DE000EC5AFD4F208301969093BB028093BA0278
:101DF000DF91CF911F910F91FF90EF90DF90CF90E7
:101E000008958091C402843009F474C0853040F490
:101E1000823001F1833058F5813009F09AC00DC04D
:101E2000863009F47FC0863008F472C0873009F428
:101E30007DC0883009F08DC085C08091BE02909130
:101E4000BF02892B09F485C08091F0018093C20202
:101E500082E075C08091BE029091BF02029708F4A3
:101E600078C08091F1018093C30283E068C08091C3
:101E7000C302863081F0873038F4833061F08530DA
:101E800051F0813011F507C0803141F08B32B9F04B
:101E90008F30D9F403C085E090E013C087E090E074
:101EA0009093BB028093BA028091BE029091BF02D0
:101EB000079758F08091F60190E0079602C084E001
:101EC00090E09093BB028093BA022091BE023091C1
:101ED000BF028091BA029091BB0282179307C8F5A6
:101EE00084E08093C4028EEB91E06BE171E00E948C
:101EF000F30F08952091BE023091BF028091BA0283
:101F00009091BB0202968217930718F585E017C0DF
:101F10000E94560C892B91F08091C202813071F49D
:101F200086E00DC00E94ED0C87E009C06091BA0206
:101F30007091BB0284E592E00E94C50188E0809325
:101F4000C40208951092BF021092BE0281E08093F5
:101F5000C402089597FB092E07260AD077FD04D006
:101F60002ED006D000201AF4709561957F4F089509
:101F7000F6F7909581959F4F0895A1E21A2EAA1B1E
:101F8000BB1BFD010DC0AA1FBB1FEE1FFF1FA21729
:101F9000B307E407F50720F0A21BB30BE40BF50B26
:101FA000661F771F881F991F1A9469F760957095AF
:101FB000809590959B01AC01BD01CF010895AA1BAE
:101FC000BB1B51E107C0AA1FBB1FA617B70710F024
:101FD000A61BB70B881F991F5A95A9F78095909556
:101FE000BC01CD010895FB01DC0101900D920020A0
:101FF000E1F708950F931F93CF93DF938C01EB01CB
:10200000009731F46115710519F420E030E038C013
:1020100081E090E06EE070E00E944712FC019C01BC
:10202000009771F180E88383209771F0D387C2878E
:1020300081E883838091C5029091C602892B21F4A7
:10204000F093C602E093C50201151105C9F011878E
:1020500000878381826083838091C7029091C80248
:10206000892B71F4F093C802E093C7028091C902F2
:102070009091CA02892B21F4F093CA02E093C9021D
:10208000C901DF91CF911F910F910895AEE0B0E0AB
:10209000ECE4F0E10C941D140D891E8986E08C831C
:1020A0001A8309838FEF9FE79E838D839E01275EAE
:1020B0003F4FCE0101966F89788DA9010E946A1069
:1020C0002F813885020F131FF80110822E96E4E04D
:1020D0000C943914ABE0B0E0E0E7F0E10C940F149D
:1020E0003C012B015A01FC0117821682838181FD7C
:1020F00003C06FEF7FEFC6C19AE0892E1E010894DE
:10210000211C311CF3012381F20123FD859123FF62
:1021100081912F01882309F4B2C1853239F423FD5E
:10212000859123FF81912F01853229F490E0B3013D
:102130000E948513E7CF982FFF24EE249924FFE116
:10214000FF15D0F09B3269F09C3228F4903259F0A0
:10215000933291F40EC09D3249F0903369F441E01E
:1021600024C052E0F52A84E0F82A28C098E0F92A31
:1021700025C0E0E1FE2A22C0F7FC29C0892F805348
:102180008A3070F4F6FE05C0989C902C1124980EAD
:1021900015C0E89CE02C1124E80EF0E2FF2A0EC0E6
:1021A0009E3229F4F6FC6BC140E4F42A07C09C3649
:1021B00019F450E8F52A02C0983649F4F20123FDDB
:1021C000959123FF91912F01992309F0B8CF892F81
:1021D0008554833018F08052833038F444E050E066
:1021E000A40EB51E5FE359830FC0933631F09337C9
:1021F00079F0933509F056C020C0F50180818983BC
:1022000042E050E0A40EB51E610101E010E012C0F2
:10221000F501C080D180F6FC03C06FEF7FEF02C0F4
:10222000692D70E042E050E0A40EB51EC6010E9488
:102230007A138C015FE7F52214C0F501C080D180CC
:10224000F6FC03C06FEF7FEF02C0692D70E042E043
:1022500050E0A40EB51EC6010E9468138C0150E820
:10226000F52AF3FE07C01AC080E290E0B3010E9495
:102270008513EA948E2D90E008171907A8F30EC075
:10228000F601F7FC8591F7FE81916F0190E0B301B3
:102290000E948513E110EA940150104001151105C8
:1022A00079F7EAC0943611F0993669F5F7FE08C05F
:1022B000F501208131814281538184E090E00AC0A0
:1022C000F501808191819C01442737FD4095542F71
:1022D00082E090E0A80EB91E9FE6F92257FF09C0E0
:1022E00050954095309521953F4F4F4F5F4FE0E817
:1022F000FE2ACA01B901A1012AE030E00E94B1130F
:10230000D82ED21840C0953729F41F2D1F7E2AE001
:1023100030E01DC01F2D197F9F3661F0903720F4EB
:10232000983509F0ACC00FC0903739F0983709F0F4
:10233000A6C004C028E030E00AC0106114FD14609B
:1023400020E130E004C014FD166020E132E017FF08
:1023500008C0F501608171818281938144E050E081
:1023600008C0F50180819181BC0180E090E042E0ED
:1023700050E0A40EB51EA1010E94B113D82ED218B0
:102380008FE7F82EF122F6FE0BC05EEFF522D9148E
:1023900038F4F4FE07C0F2FC05C08FEEF82202C04C
:1023A0001D2D01C0192DF4FE0DC0FE01ED0DF11D16
:1023B0008081803319F499EEF92208C01F5FF2FE84
:1023C00005C003C08F2D867809F01F5F0F2DF3FC29
:1023D00014C0F0FE0FC01E1510F09D2C0BC09D2CDC
:1023E0009E0C911A1E2D06C080E290E0B3010E945F
:1023F00085131F5F1E15C0F304C01E1510F4E11AEB
:1024000001C0EE2404FF0FC080E390E0B3010E94FE
:10241000851302FF1DC001FD03C088E790E00EC0D8
:1024200088E590E00BC0802F867891F001FF02C014
:102430008BE201C080E2F7FC8DE290E0B3010E94E4
:10244000851306C080E390E0B3010E9485139A943F
:10245000D914C0F3DA94F101ED0DF11D808190E003
:10246000B3010E948513DD20A9F706C080E290E049
:10247000B3010E948513EA94EE20C1F743CEF30125
:1024800066817781CB012B96E2E10C942B140F939C
:102490001F93CF93DF93689F8001699F100D789FF2
:1024A000100D1124C8010E946312EC01009729F05D
:1024B00060E070E0A8010E947313CE01DF91CF911C
:1024C0001F910F910895CF93DF93BC018230910546
:1024D00010F462E070E0A091CD02B091CE02ED0167
:1024E000E0E0F0E040E050E021C08881998186176B
:1024F000970769F48A819B81309719F093838283CF
:1025000004C09093CE028093CD02FE0134C06817C0
:10251000790738F44115510519F08417950708F427
:10252000AC01FE018A819B819C01E9012097E9F6BB
:1025300041155105A9F1CA01861B970B049708F4B0
:10254000BA01E0E0F0E02AC08D919C9111978417C8
:102550009507F9F46417750781F412968D919C9193
:102560001397309719F09383828304C09093CE021F
:102570008093CD02FD0132964FC0CA01861B970B96
:10258000FD01E80FF91F6193719302978D939C935E
:1025900043C0FD01828193819C01D9011097A1F66E
:1025A0008091CB029091CC02892B41F4809127013C
:1025B000909128019093CC028093CB024091290105
:1025C00050912A014115510541F44DB75EB78091F4
:1025D000250190912601481B590B2091CB02309187
:1025E000CC0224173507B0F4CA01821B930B86175F
:1025F000970780F0AB014E5F5F4F8417950750F04F
:10260000420F531F5093CC024093CB02F9016193C8
:10261000719302C0E0E0F0E0CF01DF91CF91089527
:10262000CF93DF93009709F450C0EC0122971B82EF
:102630001A82A091CD02B091CE02109709F140E02C
:1026400050E0AC17BD0708F1BB83AA83FE012191BE
:102650003191E20FF31FAE17BF0779F48D919C9172
:102660001197280F391F2E5F3F4F39832883129609
:102670008D919C9113979B838A834115510571F429
:10268000D093CE02C093CD0220C012968D919C9122
:102690001397AD01009711F0DC01D3CFFA01D3837A
:1026A000C28321913191E20FF31FCE17DF0769F446
:1026B00088819981280F391F2E5F3F4FFA0131839E
:1026C00020838A819B8193838283DF91CF910895B8
:1026D000FC010590615070400110D8F780959095ED
:1026E0008E0F9F1F0895DC0101C06D934150504033
:1026F000E0F70895FC016150704001900110D8F797
:10270000809590958E0F9F1F08950F931F93CF93E1
:10271000DF938C01EB018B8181FF1BC082FF0DC019
:102720002E813F818C819D812817390764F4E881CF
:10273000F9810193F983E88306C0E885F985802F44
:102740000995892B31F48E819F8101969F838E8319
:1027500002C00FEF1FEFC801DF91CF911F910F91C2
:102760000895FA01AA27283051F1203181F1E89427
:102770006F936E7F6E5F7F4F8F4F9F4FAF4FB1E074
:102780003ED0B4E03CD0670F781F891F9A1FA11D6F
:10279000680F791F8A1F911DA11D6A0F711D811D70
:1027A000911DA11D20D009F468943F912AE0269F35
:1027B00011243019305D3193DEF6CF010895462F94
:1027C0004770405D4193B3E00FD0C9F7F6CF462F75
:1027D0004F70405D4A3318F0495D31FD40524193DE
:1027E00002D0A9F7EACFB4E0A6959795879577959B
:1027F0006795BA95C9F700976105710508959B0122
:10280000AC010A2E06945795479537952795BA95AA
:10281000C9F7620F731F841F951FA01D08952F9283
:102820003F924F925F926F927F928F929F92AF9260
:10283000BF92CF92DF92EF92FF920F931F93CF93AD
:10284000DF93CDB7DEB7CA1BDB0B0FB6F894DEBF44
:102850000FBECDBF09942A88398848885F846E846A
:102860007D848C849B84AA84B984C884DF80EE80B4
:10287000FD800C811B81AA81B981CE0FD11D0FB6BD
:10288000F894DEBF0FBECDBFED010895F894FFCFE1
:10289000432533642C2534642C2534642C2534647E
:1028A0002C2534642C2533640000380A0D646164DF
:0C28B0006F733A20002000D302000000EB
:00000001FF
